:020000040000FA
:04000000A8EF17F05E
:04000800BAEF1AF041
:0400180001EF1AF0EA
:06002A0000C0E5FF01C06B
:10003000E5FF02C0E5FF03C0E5FF04C0E5FF05C022
:10004000E5FF06C0E5FF07C0E5FF08C0E5FF09C002
:10005000E5FF0AC0E5FF0BC0E5FF0CC0E5FF0201AC
:100060002351D8B492EF04F002012E972E9524C2AA
:1000700000F0010E016EC0C602F00250230A02E039
:10008000E8EF02F0020E005CD8A092EF04F0C1C6C7
:1000900002F00250530A01E07DD00050040A02E051
:1000A00092EF04F0C2C602F00250036ED00E032499
:1000B000026E0A0E025C05E30250036EF90E032481
:1000C000026EC3C603F00350046ED00E0424036E08
:1000D0000A0E035C05E30350046EF90E0424036E5C
:1000E000100E025CD8B092EF04F0100E035CD8B092
:1000F00092EF04F00238F00B046E03500426045013
:10010000D8B492EF04F0800E045CD8B092EF04F003
:100110000438E8441F0B056EC00E0524066E076AFE
:10012000000E072206C0E9FF07C0EAFFEFCF08F084
:10013000070E0414096E010E0A6E095005E0E86C02
:10014000D8900A36010FFDE30A50081206C0E9FFF5
:1001500007C0EAFF08C0EFFF066AD00E0526000EB2
:10016000062205C0E9FF06C0EAFFEFCF07F00A1E2E
:100170000A50071605C0E9FF06C0EAFF07C0EFFFF7
:10018000045002012B5DD8B092EF04F004C02BF2B2
:1001900092EF04F00250430A01E074D00050040AC8
:1001A00002E092EF04F0C2C602F00250056ED00EDB
:1001B0000524026E0A0E025C05E30250056EF90E7C
:1001C0000524026EC3C603F00350056ED00E05244D
:1001D000036E0A0E035C05E30350056EF90E052459
:1001E000036E100E025CD8B092EF04F0100E035CA8
:1001F000D8B092EF04F00238F00B0324046E0450E0
:10020000D8B492EF04F0800E045CD8B092EF04F002
:100210000438E8441F0B056ED00E0524066E076AED
:10022000000E072206C0E9FF07C0EAFFEFCF08F083
:10023000070E0414096E010E0A6E095005E0E86C01
:10024000D8900A36010FFDE30A1C096E081606C095
:10025000E9FF07C0EAFF08C0EFFF066AC00E0526E7
:10026000000E062205C0E9FF06C0EAFFEFCF07F047
:100270000750091605C0E9FF06C0EAFF09C0EFFFF5
:1002800092EF04F00250690A0EE1000EE56E240EB2
:10029000E56ED80EE56E2CEC19F0030EE12650EC5D
:1002A00017F092EF04F002504C0A01E091D0000EDA
:1002B000E56E240EE56EEA0EE56E2CEC19F0030EE9
:1002C000E12625C207F0020EE56E2E0EE56EE56A08
:1002D0000750E56E000EE56E240EE56EFC0EE56E31
:1002E0002CEC19F0070EE126056A010E066E065089
:1002F00002012B5DD8A065D00638E8441F0B076EBD
:10030000C00E0724086E096A000E092208C0E9FF22
:1003100009C0EAFFEFCF08F0070E0614096E010EC0
:100320000A6E0B6A095006E0E86CD8900A360B3664
:10033000010FFCE30C6A0A5008160B500C1608500B
:100340000C10D8B43CD0086AD00E0726000E082244
:1003500007C0E9FF08C0EAFFEFCF07F0086A0750BF
:100360000A1608500B160A500B10D880E866D89071
:100370000A6A0A360A50D880E866D8900A6A0A36AD
:10038000076A0ABE076806C008F00750E56E0A5003
:10039000E56EE56A0850E56E000EE56E250EE56E29
:1003A000220EE56E2CEC19F0070EE126052A055009
:1003B0000F0B05E10A0EE56E1BEC1CF0E652062A57
:1003C00096D70A0EE56E1BEC1CF0E65292EF04F095
:1003D0000250460A14E102012E990201256BAB98E6
:1003E0008B809D9A9D98000EE56E250EE56E2A0E77
:1003F000E56E2CEC19F0030EE12692EF04F00250AA
:10040000560A0CE1000EE56E250EE56E420EE56E15
:100410002CEC19F0030EE12692EF04F00250520A80
:1004200001E044D0000EE56A0DEC1CF0046EE652CB
:100430000F0E0414056E0A0E055C08E205C006F0F6
:10044000076A300E0626D8B0072A07D0086A05507A
:10045000370F066E000E0820076E04380F0B056E6E
:100460000A0E055C08E205C008F0096A300E08268D
:10047000D8B0092A07D00A6A0550370F086E000E57
:100480000A20096E0750E56E0650E56E0950E56ECC
:100490000850E56E000EE56E250EE56E7C0EE56EED
:1004A0002CEC19F0070EE12692EF04F00250570AE7
:1004B00034E1C2C602F00250056ED00E0524026E71
:1004C0000A0E025C05E30250056EF90E0524026E69
:1004D000C3C603F00350056ED00E0524036E0A0E4A
:1004E000035C05E30350056EF90E0524036E100E40
:1004F000025CD8B092EF04F0100E035CD8B092EF1B
:1005000004F00238F00B0324E56E000EE56A15ECEA
:1005100012F0E652E65292EF04F00250450A21E151
:10052000020E056E02012451055C14E205C006F0BE
:10053000052A076AC00E0626060E072206C0E9FF36
:1005400007C0EAFFEFCF02F00250E56E1BEC1CF093
:10055000E652E8D70A0EE56E1BEC1CF0E65292EF6D
:1005600004F00250440A02E092EF04F00050040A42
:1005700002E092EF04F0C2C602F00250056ED00E07
:100580000524026E0A0E025C05E30250056EF90EA8
:100590000524026EC3C603F00350056ED00E052479
:1005A000036E0A0E035C05E30350056EF90E052485
:1005B000036E100E025CD8B0B5D1100E035CD8B03B
:1005C000B1D10238F00B0324046E04C029F2AAD181
:1005D0000250210A01E03DD00006010E005CD8A0C7
:1005E000A1D1010E0201306F0001606B0201316B7D
:1005F000C1C602F00250420A0FE00250490A0CE064
:1006000002504E0A09E00250520A06E00250500A17
:1006100003E00250460A15E102012E850250460A07
:100620000DE102012E89000EE56E250EE56E860EA7
:10063000E56E2CEC19F0030EE126ABD002012E99E9
:10064000A8D00250620A01E06DD1020E016E0006D0
:10065000A0D002012EA958D00028056E0001606FBD
:1006600005C031F20250616F02013127020E020112
:10067000306F010E056E02012451055C21E2600E0F
:1006800002013025066E076A000E072205C008F039
:10069000052A096AC00E0826060E092208C0E9FFCD
:1006A00009C0EAFFEFCF08F006C0E9FF07C0EAFF84
:1006B00008C0EFFF0850020131270201302BDBD7C1
:1006C000600E02013025056E066A000E0622020148
:1006D000311D076E072A05C0E9FF06C0EAFF07C003
:1006E000EFFF020130290201326F0201336BAB9838
:1006F0008B909D9A60C0ADFF010E0201306F040E19
:100700000201256F9D880ED1030E005CD8A00AD18E
:100710000250056ED00E0524026E0A0E025C05E33F
:100720000250056EF90E0524026E020E016EC1C65E
:1007300003F00350056ED00E0524036E0A0E035C11
:1007400005E30350056EF90E0524036E100E025CDE
:10075000D8B0E8D0100E035CD8B0E4D00238F00B6B
:100760000324046E04AE03D002012E8502D00201E0
:100770002E95049E0450D8B4D5D0010E0201306FDE
:1007800004500001606F04C031F2FE0E0026020129
:100790002E8702012EA502D0008E02D0D890003202
:1007A000600E02013025046E056A000E052204C0A9
:1007B000E9FF05C0EAFF00C0EFFF0050020131274A
:1007C0000201302B02012EA528D001C000F0020149
:1007D0002451005CD8B07FD0600E02013025046E39
:1007E000056A000E052200C006F0002A076AC00E46
:1007F0000626060E072206C0E9FF07C0EAFFEFCF74
:1008000006F004C0E9FF05C0EAFF06C0EFFF06508E
:10081000020131270201302BDAD702012451015C99
:10082000D8B059D001C000F0012A046AC00E0026D9
:10083000060E042200C0E9FF04C0EAFFEFCF02F079
:100840000250006ED00E0024026E0A0E025C05E318
:100850000250006EF90E0024026E02012451015C68
:10086000D8B060D001C000F0012A046AC00E002692
:10087000060E042200C0E9FF04C0EAFFEFCF03F038
:100880000350006ED00E0024036E0A0E035C05E3D5
:100890000350006EF90E0024036E100E025CD8B0F7
:1008A00041D0100E035CD8B03DD00238F00B0326C7
:1008B000600E02013025006E026A000E022200C0A6
:1008C000E9FF02C0EAFF03C0EFFF03500201312736
:1008D0000201302BA2D7600E02013025006E016AA2
:1008E000000E01220201311D026E022A00C0E9FF42
:1008F00001C0EAFF02C0EFFF020130290201326F9E
:100900000201336BAB988B909D9AAC8060C02FF244
:1009100060C0ADFFAC90010E0201306F020E02010B
:10092000256F9D880201246B0201236BE4CF0CF03C
:10093000E4CF0BF0E4CF0AF0E4CF09F0E4CF08F005
:10094000E4CF07F0E4CF06F0E4CF05F0E4CF04F005
:10095000E4CF03F0E4CF02F0E4CF01F0E4CF00F005
:100960001200D9CFE5FFE1CFD9FF00C0E5FF01C0FC
:10097000E5FF02C0E5FF03C0E5FF04C0E5FF05C0D9
:10098000E5FF06C0E5FF07C0E5FF08C0E5FF09C0B9
:10099000E5FF0AC0E5FF0BC0E5FF0CC0E5FF0DC099
:1009A000E5FF0EC0E5FF0FC0E5FF10C0E5FF11C079
:1009B000E5FF12C0E5FF13C0E5FF14C0E5FF15C059
:1009C000E5FF16C0E5FF17C0E5FF18C0E5FF19C039
:1009D000E5FF1AC0E5FF1BC0E5FF1CC0E5FF1DC019
:1009E000E5FF1EC0E5FF020EDBCF00F0030EDBCFFC
:1009F00001F0040EDBCF02F0050EDBCF03F0060E94
:100A0000DBCF04F0070EDBCF05F0080EDBCF06F0DE
:100A1000090EDBCF07F00A0EDBCF08F0096A0A6A7D
:100A200002C00DF00D50800A0DE1025002010B6F63
:100A300001500A6F0050096F020E016E090E006E20
:100A4000800E026E03C0E9FF04C0F3FF05509FEC67
:100A50001BF00B6E0B50D8B467EF08F00B50250A53
:100A600002E04EEF08F00C6A0D6A0E6A0F6A106A17
:100A70000A0E116E126A136A146A200E156E166839
:100A8000176A2B0E186E032A02E3044A052A03C0D4
:100A9000E9FF04C0F3FF05509FEC1BF0196E250A17
:100AA00013E11950E56E0250E56E0150E56E0050FD
:100AB000E56E3CEC15F0040EE126094A0A2A032AE9
:100AC00002E3044A052ABED71950300A06E1300E67
:100AD000156E032A02E3044A052A03C0E9FF04C095
:100AE000F3FF05509FEC1BF02D0A06E1010E146E7A
:100AF000032A02E3044A052A03C0E9FF04C0F3FF06
:100B000005509FEC1BF0200A08E1010E176E200E25
:100B1000186E032A02E3044A052A03C0E9FF04C051
:100B2000F3FF05509FEC1BF02B0A06E1010E176E38
:100B3000032A02E3044A052A03C0E9FF04C0F3FFC5
:100B400005509FEC1BF0196E310E195C2BE33A0E29
:100B5000195C28E203C019F004C01AF005C01BF0AC
:100B600019C0E9FF1AC0F3FF1B509FEC1BF01C6E6D
:100B7000300E1C5C11E33A0E1C5C0EE213500A0DA1
:100B8000F3CF1DF01D501C26D00E1C24136E192A05
:100B900002E31A4A1B2AE4D719C003F01AC004F072
:100BA0001BC005F003C0E9FF04C0F3FF05509FEC34
:100BB0001BF02E0A2DE1032A02E3044A052A166AD5
:100BC00003C019F004C01AF005C01BF019C0E9FFFA
:100BD0001AC0F3FF1B509FEC1BF01C6E300E1C5C08
:100BE00011E33A0E1C5C0EE216500A0DF3CF1DF015
:100BF0001D501C26D00E1C24166E192A02E31A4A18
:100C00001B2AE4D719C003F01AC004F01BC005F07A
:100C100003C0E9FF04C0F3FF05509FEC1BF0196E01
:100C20006C0A07E1010E0C6E032A02E3044A052A4E
:100C300009D01950680A06E1010E0E6E032A02E37C
:100C4000044A052A03C0E9FF04C0F3FF05509FECE6
:100C50001BF0750A06E1010E106E032A02E3044A36
:100C6000052A03C0E9FF04C0F3FF05509FEC1BF009
:100C7000196E730A05E1010E0D6E200E156E3FD040
:100C80001950780A03E1100E116E39D01950580A24
:100C900005E1100E116E010E126E31D01950630A6B
:100CA00002E1116A2CD019506F0A03E1080E116E8F
:100CB00026D01950660A03E1010E0F6E20D019509C
:100CC000640A1DE01950690A1AE0105005E0FF0E91
:100CD00003260422052213D01950E56E0250E56E5A
:100CE0000150E56E0050E56E3CEC15F0040EE12677
:100CF000094A0A2A032A02E3044A052AA3D60D5008
:100D000021E00650030F0D6E000E0720196E000E35
:100D100008201A6E0DC006F019C007F01AC008F0BE
:100D2000FD0E0D26FF0E19221A220DC0E9FF19C073
:100D3000F3FF1A50D5EC1AF00D6EF3CF19F0F4CF83
:100D40001AF0FDD00F500DE0000E1A6E110E196E44
:100D5000560E0D6E040E0626000E07220822166897
:100D6000EED016680C5023E00650040F0C6E000EF7
:100D700007200F6E000E08201B6E0CC006F00FC07F
:100D800007F01BC008F0FC0E0C26FF0E0F221B22E2
:100D90000CC0E9FF0FC0F3FF1B509AEC1AF00C6E69
:100DA000F3CF0FF0F4CF1BF0E9CF1CF067D00E505B
:100DB0002FE00650020F0E6E000E07201D6E000E73
:100DC00008201E6E0EC006F01DC007F01EC008F001
:100DD000FE0E0E26FF0E1D221E220EC0E9FF1DC0B4
:100DE000F3FF1E504DEC1BF00E6E0EC00CF00F6AA0
:100DF0001B6A1C6A11500A0A03E11050D8B43ED095
:100E00000C500E6E0EC00CF00F6A1B6A1C6A36D0B6
:100E10000650020F0E6E000E07201D6E000E0820F9
:100E20001E6E0EC006F01DC007F01EC008F0FE0EBC
:100E30000E26FF0E1D221E220EC0E9FF1DC0F3FF6D
:100E40001E504DEC1BF00E6EF3CF1DF00EC00CF0DB
:100E50001DC00FF0E86A1DBEFF0E1B6E1C6E115008
:100E60000A0A02E110500AE00C500E6E0F501D6E7F
:100E70000EC00CF01DC00FF01B6A1C6A000E196E2C
:100E8000E10E0D6E800E1A6E1150D8B440D0105085
:100E900013E01150E56E000EE56EE10EE56E1C509C
:100EA000E56E1B50E56E0F50E56E0C50E56E39ECAB
:100EB00011F0070EE12612D01150E56E000EE56E1E
:100EC000E10EE56E1C50E56E1B50E56E0F50E56EB1
:100ED0000C50E56E36EC16F0070EE12617502FE0A9
:100EE0000DC0E9FF19C0F3FF1A509FEC1BF02D0A4B
:100EF00026E0FF0E0D2619221A2218C0E5FF0DC0AC
:100F0000E9FF19C0F3FF1A503FEC1CF018D00CC0D9
:100F1000E5FF0DC0E9FF19C0F3FF1A503FEC1CF0CC
:100F20000D50010F0C6E000E19200E6E000E1A20CF
:100F3000E56A0CC0E9FF0EC0F3FF3FEC1CF00DC0EA
:100F40000CF019C00EF01AC00FF013C010F01050C2
:100F500010E00CC0E9FF0EC0F3FF0F509FEC1BF038
:100F6000176E175006E00C2A02E30E4A0F2A1006ED
:100F7000EED710C013F014501EE109C00CF00AC0E7
:100F80000EF010C00FF00F5010E01550E56E02503B
:100F9000E56E0150E56E0050E56E3CEC15F0040E78
:100FA000E1260C4A0E2A0F06EED70CC009F00EC03F
:100FB0000AF00FC013F016C00CF00DC00DF019C0F0
:100FC0000EF01AC00FF009C010F00AC015F00DC0E5
:100FD000E9FF0EC0F3FF0F509FEC1BF0166E16508A
:100FE000D8B43ED00CC016F0176A161E171E165045
:100FF000171005E00CC016F00C06165031E00DC0BD
:10100000E9FF0EC0F3FF0F509FEC1BF0116E125062
:1010100010E01150E56E20EC1BF0166EE6521650F3
:1010200004E0DF0E1114166E02D011C016F016C0C7
:1010300011F01150E56E0250E56E0150E56E005062
:10104000E56E3CEC15F0040EE1260D2A02E30E4A93
:101050000F2A104A152A1350D8B4B9D71306B7D798
:1010600010C009F015C00AF014502BE010C00CF0AD
:1010700015C00DF013C00EF00E501FE0200EE56EEF
:101080000250E56E0150E56E0050E56E3CEC15F047
:10109000040EE1260C4A0D2A0E06EED70B50E56E23
:1010A0000250E56E0150E56E0050E56E3CEC15F027
:1010B000040EE126094A0A2A04D00CC009F00DC02A
:1010C0000AF0032A02E3044A052A22EF05F00AC0C7
:1010D000F3FF0950E4CF1EF0E4CF1DF0E4CF1CF085
:1010E000E4CF1BF0E4CF1AF0E4CF19F0E4CF18F00E
:1010F000E4CF17F0E4CF16F0E4CF15F0E4CF14F00E
:10110000E4CF13F0E4CF12F0E4CF11F0E4CF10F00D
:10111000E4CF0FF0E4CF0EF0E4CF0DF0E4CF0CF00D
:10112000E4CF0BF0E4CF0AF0E4CF09F0E4CF08F00D
:10113000E4CF07F0E4CF06F0E4CF05F0E4CF04F00D
:10114000E4CF03F0E4CF02F0E4CF01F0E4CF00F00D
:10115000E4CFD9FF12003C4E4F20464C4F41543E45
:101160000000D9CFE5FFE1CFD9FF00C0E5FF01C006
:10117000E5FF02C0E5FF03C0E5FF04C0E5FF05C0D1
:10118000E5FF06C0E5FF07C0E5FF08C0E5FF09C0B1
:10119000E5FF0AC0E5FF0BC0E5FF0CC0E5FF0DC091
:1011A000E5FF020ED924006E000EDA20016E800EDB
:1011B000026E030E0026000E01220222020EDBCF79
:1011C00003F0030EDBCF04F0040EDBCF05F003C009
:1011D000E9FF04C0F3FF05509FEC1BF0066E0EC044
:1011E000E5FF0FC0E5FF10C0E5FF0350010F0E6ED5
:1011F000000E04200F6E000E0520106E020E0EC0B1
:10120000DBFF030E0FC0DBFF040E10C0DBFFE4CFDB
:1012100010F0E4CF0FF0E4CF0EF006C003F006505C
:10122000D8B45EEF0BF00350250A06E00350E56EDC
:101230001BEC1CF0E652C2D7046A056A020EDBCF33
:1012400006F0030EDBCF07F0040EDBCF08F006C07C
:10125000E9FF07C0F3FF08509FEC1BF0036E0EC0C0
:10126000E5FF0FC0E5FF10C0E5FF0650010F0E6E51
:10127000000E07200F6E000E0820106E020E0EC02A
:10128000DBFF030E0FC0DBFF040E10C0DBFFE4CF5B
:1012900010F0E4CF0FF0E4CF0EF00350300A31E14C
:1012A000020EDBCF06F0030EDBCF07F0040EDBCF20
:1012B00008F006C0E9FF07C0F3FF08509FEC1BF0E1
:1012C000036E0EC0E5FF0FC0E5FF10C0E5FF06503E
:1012D000010F0E6E000E07200F6E000E0820106E1C
:1012E000020E0EC0DBFF030E0FC0DBFF040E10C0AA
:1012F000DBFFE4CF10F0E4CF0FF0E4CF0EF0010EEF
:10130000046E300E035CD8A066D03A0E035CD8B0F1
:1013100062D0056A020EDBCF06F0030EDBCF07F0CA
:10132000040EDBCF08F0300E035C3AE33A0E035CA8
:1013300037E20544E844FC0B096E055009260944D0
:10134000FE0B0A6E03500A24096ED00E0924056EA6
:1013500006C0E9FF07C0F3FF08509FEC1BF0036EC7
:10136000062A02E3074A082A0EC0E5FF0FC0E5FF80
:1013700010C0E5FF06C00EF007C00FF008C010F067
:10138000020E0EC0DBFF030E0FC0DBFF040E10C009
:10139000DBFFE4CF10F0E4CF0FF0E4CF0EF0C3D7C3
:1013A0000EC0E5FF0FC0E5FF10C0E5FF06C00EF060
:1013B00007C00FF008C010F0020E0EC0DBFF030ED6
:1013C0000FC0DBFF040E10C0DBFFE4CF10F0E4CF52
:1013D0000FF0E4CF0EF0000E0201016FED0E006F72
:1013E000800E026F00C206F001C207F002C208F0D0
:1013F00002011C6B035001E161D10350250A01E198
:10140000FAD0096A0350580A01E1092A0950D8A400
:1014100072D00350630A01E1ADD00A6A0350640A36
:1014200001E10A2A0A500CE10350730A01E1C2D01B
:101430000350750A05E00350780A01E15CD0E0D062
:101440000050020F0B6E000E01200C6E000E0220E9
:101450000D6E0BC000F00CC001F00DC002F0FE0ECE
:101460000B26FF0E0C220D220B500BC0E9FF0CC007
:10147000F3FF0D504DEC1BF00201106FF3CF11F292
:101480000A5014E010510A6E11510B6ED8800BAE49
:10149000D8900CE30B1C116F0A1C106F103F01D089
:1014A000112B2D0EE56ED2EC19F0E652270EE56EEB
:1014B000100EE56E6CEC19F0E652E652030EE56E86
:1014C000E80EE56E6CEC19F0E652E652E56A640E41
:1014D000E56E6CEC19F0E652E652E56A0A0EE56E2E
:1014E0006CEC19F0E652E65202011051E56EA0ECE8
:1014F00019F0E65285D009C01BF20050020F096EA8
:10150000000E01200A6E000E02200B6E09C000F0D2
:101510000AC001F00BC002F0FE0E0926FF0E0A22DF
:101520000B2209C0E9FF0AC0F3FF0B504DEC1BF082
:101530000201106FF3CF11F2100EE56E000EE56A96
:101540006CEC19F0E652E652010EE56E000EE56A0B
:101550006CEC19F0E652E652E56A100EE56E6CECA2
:1015600019F0E652E65202011051E56EA0EC19F0B6
:10157000E65246D00050020F096E000E01200A6E9E
:10158000000E02200B6E09C000F00AC001F00BC073
:1015900002F0FE0E0926FF0E0A220B2209C0E9FF07
:1015A0000AC0F3FF0B504DEC1BF0E56ED2EC19F0C6
:1015B000E65226D00050030F096E000E01200A6E7D
:1015C000000E02200B6E09C000F00AC001F00BC033
:1015D00002F0FD0E0926FF0E0A220B2209C0E9FFC8
:1015E0000AC0F3FF0B50D5EC1AF0066EF3CF07F0EC
:1015F000F4CF08F005D0250EE56ED2EC19F0E652D6
:1016000000C209F001C20AF002C20BF0E56A09C08B
:10161000E9FF0AC0F3FF0B503FEC1CF006C000F2DC
:1016200007C001F208C002F200C209F001C20AF0CC
:1016300002C20BF009C0E9FF0AC0F3FF0B509FEC98
:101640001BF0096E0201002B03E3013F01D0022BC6
:10165000095004E0055002E00506E6D705C009F090
:10166000050609500DE0045003E0300E096E02D06B
:10167000200E096E0950E56E1BEC1CF0E652EED709
:1016800006C004F007C005F008C006F004C0E9FF7A
:1016900005C0F3FF06509FEC1BF0076E042A02E31F
:1016A000054A062A07C003F00750D8B4DEEF08F059
:1016B0000350E56E1BEC1CF0E652E8D7E4CF0DF0CA
:1016C000E4CF0CF0E4CF0BF0E4CF0AF0E4CF09F064
:1016D000E4CF08F0E4CF07F0E4CF06F0E4CF05F064
:1016E000E4CF04F0E4CF03F0E4CF02F0E4CF01F064
:1016F000E4CF00F0E4CFD9FF120000C0E5FF01C045
:10170000E5FF02C0E5FF03C0E5FF04C0E5FF05C03B
:10171000E5FF06C0E5FF07C0E5FF02012EAB0BD0D9
:101720002E9B000EE56E240EE56EC40EE56E2CECCD
:1017300019F0030EE12602012EAD0BD02E9D000EF6
:10174000E56E240EE56ECE0EE56E2CEC19F0030E60
:10175000E1260201265101E1CAD1010E0201265DF6
:10176000D8A0C3D1060E265DD8B0BFD12605006E25
:10177000FA6AFB6A0034FA36E834FA36FC0B8E0F4C
:10178000E56E170EFA22000EFB22E450F96ED1EF3F
:101790000BF048EF0CF0BFEF0CF0FCEF0CF039EF62
:1017A0000DF002012F39E8441F0B006E016AD00EC4
:1017B0000026000E012200C0E9FF01C0EAFFEFCFC2
:1017C00002F0070E2F15036E010E046E056A03501A
:1017D00006E0E86CD89004360536010FFCE302C041
:1017E00006F0076A06500416075005160450051047
:1017F000D8A47BD1010E046E035005E0E86CD890AC
:101800000436010FFDE30450021200C0E9FF01C0DD
:10181000EAFF02C0EFFF0A0EE56E1BEC1CF0E65279
:10182000730EE56E1BEC1CF0E652430EE56E1BECEE
:101830001CF0E65202012F390F0B006E0A0E005CFD
:1018400005E20050016E300E012603D0370E002451
:10185000016E0150E56E1BEC1CF0E6520F0E02010A
:101860002F15006E0A0E005C05E20050016E300E6E
:10187000012603D0370E0024016E0150E56E1BECEB
:101880001CF0E6520A0EE56E1BEC1CF0E6522DD160
:1018900002012F39E8441F0B006E016AD00E0026AA
:1018A000000E012200C0E9FF01C0EAFFEFCF02F005
:1018B000070E2F15036E010E046E056A035006E035
:1018C000E86CD89004360536010FFCE302C006F040
:1018D000076A065004160750051604500510D8B4C0
:1018E00004D1010E046E035005E0E86CD890043674
:1018F000010FFDE3041C021600C0E9FF01C0EAFF6E
:1019000002C0EFFF0A0EE56E1BEC1CF0E652730EF0
:10191000E56E1BEC1CF0E652630EE56E1BEC1CF052
:10192000E65202012F390F0B006E0A0E005C05E231
:101930000050016E300E012603D0370E0024016ED8
:101940000150E56E1BEC1CF0E6520F0E02012F1544
:10195000006E0A0E005C05E20050016E300E01269A
:1019600003D0370E0024016E0150E56E1BEC1CF015
:10197000E6520A0EE56E1BEC1CF0E652B6D00A0EDB
:10198000E56E1BEC1CF0E652730EE56E1BEC1CF0D2
:10199000E652780EE56E1BEC1CF0E65202012F3980
:1019A0000F0B006E0A0E005C05E20050016E300E57
:1019B000012603D0370E0024016E0150E56E1BECAA
:1019C0001CF0E6520F0E02012F15006E0A0E005C8D
:1019D00005E20050016E300E012603D0370E0024C0
:1019E000016E0150E56E1BEC1CF0E6520A0EE56E2E
:1019F0001BEC1CF0E65279D00A0EE56E1BEC1CF0D5
:101A0000E652730EE56E1BEC1CF0E652610EE56EBD
:101A10001BEC1CF0E65202012F390F0B006E0A0E70
:101A2000005C05E20050016E300E012603D0370E37
:101A30000024016E0150E56E1BEC1CF0E6520F0E07
:101A400002012F15006E0A0E005C05E20050016EC7
:101A5000300E012603D0370E0024016E0150E56ED2
:101A60001BEC1CF0E6520A0EE56E1BEC1CF0E65275
:101A70003CD00A0EE56E1BEC1CF0E652730EE56ED0
:101A80001BEC1CF0E652540EE56E1BEC1CF0E6520B
:101A900002012F390F0B006E0A0E005C05E20050A8
:101AA000016E300E012603D0370E0024016E015066
:101AB000E56E1BEC1CF0E6520F0E02012F15006EB6
:101AC0000A0E005C05E20050016E300E012603D0C4
:101AD000370E0024016E0150E56E1BEC1CF0E6523F
:101AE0000A0EE56E1BEC1CF0E6520201266BE4CFF9
:101AF00007F0E4CF06F0E4CF05F0E4CF04F0E4CF44
:101B000003F0E4CF02F0E4CF01F0E4CF00F01200E4
:101B100000C0E5FF01C0E5FF02C0E5FFABA202D0B7
:101B200002012E8BABA402D002012E8D02012551A1
:101B3000010A01E038D09DBA0BD09EA208D04AEC31
:101B40001CF09D921F0ECA6E6A0ECC6E9E9244D1FE
:101B50009EAA28D0030ECA6E9D929E92AECF00F030
:101B6000AB988B809D9A9D98005019E00201332B11
:101B7000030E335D11E2AB988B909D9AAC8060C0F0
:101B80002FF260C0ADFFAC90010E0201306F020E6B
:101B90000201256F9D8820D1040E0201266F0201EB
:101BA000256B1AD119D102012551030A01E068D031
:101BB0009DBA0BD09EA208D04AEC1CF09D921F0E3D
:101BC000CA6E6A0ECC6E9E9207D19EAA58D0AECF36
:101BD00000F0800E02012725016E026A060E022225
:101BE00001C0E9FF02C0EAFF00C0EFFF272B6A0E29
:101BF000CC6E9E922751010A1EE10201346B3F0E0A
:101C000000140201286F282B00500EE1030ECA6E4B
:101C10009D929E92AB988B809D9A9D980201256B18
:101C2000010E0201266F07D000AE03D002012E8301
:101C300002D002012E9300500201342702012751E5
:101C40000201285D1BE2030ECA6E9D929E92AB9824
:101C50008B809D9A9D980201256B0201345109E108
:101C60000201270702012E81010E0201266FAD6AD3
:101C700005D0030E0201266F010EAD6EADD0ACD0C3
:101C800002012551020A01E04ED09EA212D00201AB
:101C90003051020132190DE1030ECA6E9D929E92DF
:101CA0000201256B4AEC1CF0AB988B809D9A9D98A5
:101CB00093D09EB801D090D0030ECA6E9D929E9292
:101CC00030C201F00201302B026A600E0126000EC4
:101CD000022201C0E9FF02C0EAFFEFCFADFF3051A1
:101CE000020132191FE19D9802012EA70BD09D928F
:101CF000070ECA6ED00ECC6E9E929D82010E02011E
:101D0000256F10D002012EA906D04AEC1CF0050E5A
:101D10000201256F07D09D92070ECA6ED00ECC6EC1
:101D20009E929D8259D002012551040A29E1030E99
:101D3000CA6E9D929E929EA84FD030C201F00201C1
:101D4000302B026A600E0126000E022201C0E9FF5C
:101D500002C0EAFFEFCFADFF3051020132190FE1AF
:101D60009D989D92070ECA6ED00ECC6E9E929D825B
:101D7000050E0201256F0201286B0201276B2CD092
:101D800002012551050A1FE19DBA09D09EA206D085
:101D90004AEC1CF0030ECA6E9D929E921DD09EAA24
:101DA00011D0AECF00F0800E02012725016E026A2D
:101DB000060E022201C0E9FF02C0EAFF00C0EFFFE9
:101DC000272B0AD009D00201255106E1030ECA6E65
:101DD0009D929E929D989D9AE4CF02F0E4CF01F0EF
:101DE000E4CF00F0120000C0E5FF01C0E5FF02C033
:101DF000E5FF03C0E5FF6C50D8A434D13C0E0401CC
:101E00000015006E0040E8403F0B0D0A01E0EAD0EB
:101E10007F0E04010415046F7F0E0015006F020190
:101E2000176B0201186B0201196B41C500F000C06D
:101E3000FBF00050050A09E1010E0201186F040EC3
:101E400002011A6F42C514F288D00050060A03E15D
:101E500010EC14F082D00050090A2EE1010E0201AC
:101E6000186F42C515F20201155104E1040E02017A
:101E70001A6F73D0050E02011A6F1E0E716E600E7E
:101E800004010E6F040E0F6F400E04010C6F1E0E46
:101E9000726E400E0401116F000E126F050E136F6B
:101EA000880E0401106F200E0401166F040E176FC8
:101EB000400E0401146F51D00050080A12E1010EC7
:101EC0000201186F1A0E020115250001FD6FFE6B4D
:101ED000300EFE23FF6B000EFF23010E0201196F6F
:101EE0003CD0005003E1C5EC15F037D00050010A9A
:101EF00003E00050030A03E1F6EC16F02ED0005088
:101F00000A0A0EE1010E0201186F180E0001FD6FA2
:101F1000300EFE6F000EFF6F010E0201196F1DD013
:101F200000500B0A06E00050200A03E00050220A8D
:101F300004E1010E0201186F10D00050210A0DE1DA
:101F4000960E0001FD6F300EFE6F000EFF6F070E44
:101F50000201196F010E0201186F020118510CE104
:101F6000100E0401016F400E026F050E036F840E08
:101F70000401006F046F34D0050140AF1FD019C2B7
:101F800000F0016A0150475D02E10050465D04E245
:101F9000050146510201196F99EC16F0020E02017B
:101FA000176F100E0401016F400E026F050E036FD4
:101FB000800E0401006FC80E046F12D0010E0201E2
:101FC000176F0401056BC80E0401046F100E0401A5
:101FD000016F800E026F050E036FC80E0401006FC3
:101FE0006D9862D002011751010A01E038D0040156
:101FF000015102011927800E02010C6F050E0D6FB1
:1020000001C416F216C200F00201160700501DE0CE
:102010000EC200F00FC201F00CC202F00DC203F0BC
:1020200002C0E9FF03C0EAFFEFCF02F002010C3F5C
:1020300001D00D2B00C0E9FF01C0EAFF02C0EFFF95
:1020400002010E3F01D00F2BDDD7040100AD03D0FC
:10205000880E006F29D0C80E0401006F25D0E0EC77
:102060001BF022D06C50040A1FE16E500BE10201FC
:102070001A51040A07E142C56EFF6E5003E1030ED8
:1020800002011A6F02011751020A0CE199EC16F0D5
:10209000040104AD03D0880E046F06D0C80E0401FD
:1020A000046F02D0E0EC1BF0E4CF03F0E4CF02F0C9
:1020B000E4CF01F0E4CF00F0120000C0E5FF01C062
:1020C000E5FF7DEC0BF002012551050A28E1020134
:1020D0002751020128191CE0020127510201281989
:1020E00015E028C200F00201282B016A800E0026AC
:1020F000060E012200C0E9FF01C0EAFFEFCF00F0A9
:102100000050E56E1BEC1CF0E652E6D75BEC1CF0D1
:1021100002012351D8B4A5D015EC00F0A2D0F29E54
:1021200002012551D8A45DD0030ECA6E9D929E92E5
:102130000201235103E015EC00F093D002012EB10F
:1021400090D0020129510201355DD8A08AD0356BAB
:1021500002012C2B2C5102012B5D07E2010E020122
:102160002C6F020E02012D6F03D002012D352D3789
:1021700002012C39E8441F0B006E016AC00E0026D4
:10218000000E012200C0E9FF01C0EAFFEFCF00F01E
:1021900002012D5100160050D8B463D00201286B03
:1021A0000201276B0201346BAC80AB988B909D9A37
:1021B0007DEC0BF0F29C2CC22FF2800E02012C1150
:1021C000AD6EAC90800E2C11AD6E9D92070ECA6E56
:1021D000D00ECC6E9E929D82030E0201256FF28C72
:1021E00040D002012551010A27E19DAA3AD09EA2C2
:1021F00038D0030ECA6E9D929E92AB988B809D9AAA
:102200009D980201332B335D11E2AB988B909D9A20
:10221000AC8060C02FF260C0ADFFAC90010E020137
:10222000306F020E0201256F9D881BD0050E020142
:10223000266F0201256B15D002012551030A11E119
:102240009DAA0FD09EA20DD0030ECA6E9D929E92A3
:10225000020E0201266FAB988B809D9A9D98020119
:10226000256BF28ECFEC12F0E4CF01F0E4CF00F05A
:102270001200D9CFE5FFE1CFD9FF00C0E5FF01C0D3
:10228000E5FF02C0E5FF03C0E5FF04C0E5FF05C0B0
:10229000E5FF06C0E5FF07C0E5FF08C0E5FF09C090
:1022A000E5FF0AC0E5FF0BC0E5FF0CC0E5FF0DC070
:1022B000E5FF0EC0E5FF0FC0E5FF020EDBCF00F02B
:1022C000030EDBCF01F0040EDBCF02F0050EDBCFF7
:1022D00003F0060EDBCF04F0070EDBCF05F0080E8F
:1022E000DBCF06F0200E076E086A06C009F00A6A06
:1022F0000B6A0C6AE56AE56AE56A0950E56E035007
:10230000E56E0250E56E0150E56E0050E56E73EC2F
:1023100013F00D6E080EE126300E0D263A0E0D5C00
:1023200005E30D500E6E270E0E240D6EFF0E0726D0
:102330000822A00E07240E6E000E08200F6E0EC09D
:10234000E9FF0FC0EAFF0DC0EFFF0C50E56E0B5028
:10235000E56E0A50E56E0950E56E0350E56E0250D9
:10236000E56E0150E56E0050E56EACEC14F0006EC9
:10237000F3CF01F0F4CF02F0E9CF03F0080EE1262D
:102380000050011002100310D8A4AFD707C000F00E
:1023900008C001F004C002F005C003F000C004F062
:1023A00001C005F0004A012AA00E0426000E0522F5
:1023B00004C0E9FF05C0EAFFEFCF04F002C0E9FF67
:1023C00003C0EAFF04C0EFFF024A032A000E015CCB
:1023D00002E1200E005CE2E302C0E9FF03C0EAFF75
:1023E000000EEF6AE4CF0FF0E4CF0EF0E4CF0DF073
:1023F000E4CF0CF0E4CF0BF0E4CF0AF0E4CF09F027
:10240000E4CF08F0E4CF07F0E4CF06F0E4CF05F026
:10241000E4CF04F0E4CF03F0E4CF02F0E4CF01F026
:10242000E4CF00F0E4CFD9FF1200D9CFE5FFE1CF30
:10243000D9FF00C0E5FF01C0E5FF02C0E5FF020EC5
:10244000DBCF00F0030EDBCFA8FF00C0A9FFA69EE4
:10245000A69CA684F29E550EA76EAA0EA76EA68213
:10246000A6A202D00000FCD7A6A610D0000E026ED5
:10247000240E016EA20E006E0250E56E0150E56E54
:102480000050E56E2CEC19F0030EE126A694F28EB6
:10249000E4CF02F0E4CF01F0E4CF00F0E4CFD9FFC5
:1024A00012004552524F523A2077726974696E6732
:1024B00020746F20454550524F4D206661696C6510
:1024C00064210A004F4552522021210A000046454E
:1024D00052522021210A00007320667261697365DF
:1024E00020696E69742E2E2E0A000A7320667261AE
:1024F000697365206C6F67203A0A00004672616953
:1025000073655374617465203A202564203B20462E
:1025100072616973655374617475733A2025640A36
:10252000000025643A25642000005175697420621A
:102530006F6F746C6F61646572206D6F64652E0AD5
:1025400000007356205573624672616973652032CC
:102550002E312E352028537061726554696D654C9B
:102560006162732F534443432920412E526F757388
:102570007365617520323031360A00007349442595
:102580006325630A0000456E74657220626F6F7484
:102590006C6F61646572206D6F64652E0A0000C007
:1025A000E5FF01C0E5FF02C0E5FF03C0E5FF020152
:1025B0002EA190D002012C390F0B006E02012EB318
:1025C00000860050016E300E0124006E3A0E005C51
:1025D00005E30050016E070E0124006E0050E56E09
:1025E0001BEC1CF0E6520F0E02012C15016E300E92
:1025F0000124006E3A0E005C05E30050016E070EE8
:102600000124006E0050E56E1BEC1CF0E652020146
:102610002EA31BD0010E016E02012751015CD8B020
:102620004ED001C002F0012A036A800E0226060E77
:10263000032202C0E9FF03C0EAFFEFCF02F002501D
:10264000E56E1BEC1CF0E652E7D7010E016E0201AD
:102650002751015C34E201C002F0012A036A800EB6
:102660000226060E032202C0E9FF03C0EAFFEFCFF5
:1026700002F002380F0B036E300E0324006E3A0E88
:10268000005C05E30050036E070E0324006E00504B
:10269000E56E1BEC1CF0E6520F0E0216300E022403
:1026A000006E3A0E005C05E30050026E070E022435
:1026B000006E0050E56E1BEC1CF0E652C8D70A0E07
:1026C000E56E1BEC1CF0E6520201276B0201286B41
:1026D00002012E91E4CF03F0E4CF02F0E4CF01F049
:1026E000E4CF00F01200D9CFE5FFE1CFD9FF00C061
:1026F000E5FF01C0E5FF02C0E5FF03C0E5FF04C040
:10270000E5FF05C0E5FF06C0E5FF07C0E5FF08C01F
:10271000E5FF09C0E5FF0AC0E5FF020EDBCF00F0D0
:10272000030EDBCF01F0040EDBCF02F0050EDBCF92
:1027300003F0060EDBCF04F0070EDBCF05F0080E2A
:10274000DBCF06F0090EDBCF07F0086A0450051056
:102750000610071005E1E968F468F368E86847D0F7
:10276000096A0750800BE8440A6E0A501BE10450C6
:1027700004260536063607360750035C08E1065086
:10278000025C05E10550015C02E10450005C06E2D8
:10279000D890073206320532043204D0092A09C023
:1027A00008F0DFD70750035C08E10650025C05E142
:1027B0000550015C02E10450005C08E30450005E37
:1027C0000550015A0650025A0750035AD890073252
:1027D00006320532043208C009F008060950E2E169
:1027E00003C0E9FF02C0F4FF01C0F3FF0050E4CFD3
:1027F0000AF0E4CF09F0E4CF08F0E4CF07F0E4CF2B
:1028000006F0E4CF05F0E4CF04F0E4CF03F0E4CF2A
:1028100002F0E4CF01F0E4CF00F0E4CFD9FF1200E2
:1028200000C0E5FF01C0E5FF02C0E5FF03C0E5FF12
:1028300004C0E5FF05014051800A01E082D043C594
:1028400000F042C501F00050010A1AE1010E020138
:10285000186FFC0E0001FD6F2F0EFE6F000EFF6F54
:10286000FDC002F0FEC003F0FFC004F002C0F6FF9E
:1028700003C0F7FF04C0F8FF0900F5CF19F261D0DB
:102880000050060A0EE1010E0201186F0E0E000143
:10289000FD6F300EFE6F000EFF6F0A0E0201196F02
:1028A00050D00050020A1CE1010E0201186F000E08
:1028B0000001FF6F300EFE6F200EFD6F020F026EE3
:1028C000000EFE21036E000EFF21046E02C0F6FF13
:1028D00003C0F7FF04C0F8FF0900F5CF19F231D0AB
:1028E0000050030A2EE1010E0201186F015008E1A9
:1028F000640E0001FD6F300EFE6F000EFF6F12D0F0
:102900000150010A08E1680E0001FD6F300EFE6FF4
:10291000000EFF6F07D0760E0001FD6F300EFE6FC8
:10292000000EFF6FFDC000F0FEC001F0FFC002F01E
:1029300000C0F6FF01C0F7FF02C0F8FF0900F5CFA5
:1029400019F2E4CF04F0E4CF03F0E4CF02F0E4CFD7
:1029500001F0E4CF00F01200D9CFE5FFE1CFD9FFBD
:1029600000C0E5FF01C0E5FF02C0E5FF03C0E5FFD1
:1029700004C0E5FF05C0E5FF06C0E5FF07C0E5FFB1
:1029800008C0E5FF09C0E5FF0AC0E5FF0BC0E5FF91
:102990000CC0E5FF0DC0E5FF020EDBCF00F0030E1B
:1029A000DBCF01F0040EDBCF02F0050EDBCF03F02E
:1029B000060EDBCF04F0070EDBCF05F0080EDBCFF1
:1029C00006F0090EDBCF07F0086A096A0A6A0B6A8B
:1029D000200E0C6E0350800BE8440D6E0050002654
:1029E0000136023603360850082609360A360B36F9
:1029F0000D50D8A4088007500B5C08E106500A5C13
:102A000005E10550095C02E10450085C09E304504B
:102A1000085E0550095A06500A5A07500B5A0080A2
:102A20000C040D6E0DC00CF00D50D4E103C0E9FF95
:102A300002C0F4FF01C0F3FF0050E4CF0DF0E4CF7B
:102A40000CF0E4CF0BF0E4CF0AF0E4CF09F0E4CFD0
:102A500008F0E4CF07F0E4CF06F0E4CF05F0E4CFD0
:102A600004F0E4CF03F0E4CF02F0E4CF01F0E4CFD0
:102A700000F0E4CFD9FF1200D9CFE5FFE1CFD9FFB5
:102A800000C0E5FF01C0E5FF02C0E5FF03C0E5FFB0
:102A900004C0E5FF05C0E5FF06C0E5FF07C0E5FF90
:102AA000020EDBCF00F0030EDBCF01F0040EDBCF14
:102AB00002F0050EDBCF03F002C006F00650046EF4
:102AC000800A33E100C0E9FF01C0F3FF0250D5ECFA
:102AD0001AF0056EF3CF06F0F4CF07F003C0E5FF60
:102AE00005C0E9FF06C0F3FF07503FEC1CF000C033
:102AF000E9FF01C0F3FF0250D5EC1AF0056EF3CFE9
:102B000006F0F4CF07F0052A02E3064A072A05C0BB
:102B1000E5FF06C0F4FF07C0F6FF00C0E9FF01C0F3
:102B2000F3FF0250FEEC1BF01DD004AA1BD0047A68
:102B3000045004E1035069EC1CF014D00450010A65
:102B400004E1035072EC1CF00DD004500F0A04E1B4
:102B500003501BEC1CF006D004500E0A03E1035096
:102B60006DEC1CF0E4CF07F0E4CF06F0E4CF05F005
:102B7000E4CF04F0E4CF03F0E4CF02F0E4CF01F0BF
:102B8000E4CF00F0E4CFD9FF120000C0E5FF01C0A0
:102B9000E5FF02C0E5FF03C0E5FF04C0E5FF1F0E2F
:102BA00005014015006E00500BE1010E0201186F87
:102BB0001E0E0001FD6F300EFE6F000EFF6F45D040
:102BC0000050010A0BE1180E0001FD6F300EFE6F80
:102BD000000EFF6F010E0201186F37D00050020A7D
:102BE00034E10F0E05014415006E800E4415016E90
:102BF000010E0201186F000E026E040E036E0050EB
:102C0000080DF450046EF3CF00F0005002240201CE
:102C10000E6F045003200F6F015004E0040E0E27C6
:102C200001E30F2B0EC200F00FC201F000C0E9FF5C
:102C300001C0EAFFEFCF00F000A407D01C0E000196
:102C4000FD6F300EFE6F000EFF6F0201185103E0A2
:102C5000020E0201196FE4CF04F0E4CF03F0E4CFD9
:102C600002F0E4CF01F0E4CF00F01200D9CFE5FF8D
:102C7000E1CFD9FF00C0E5FF01C0E5FF02C0E5FFDD
:102C800003C0E5FF04C0E5FF05C0E5FF06C0E5FFA2
:102C9000020EDBCF00F0030EDBCF01F0040EDBCF22
:102CA00002F0050EDBCF03F0060EDBCF04F0070EBB
:102CB000DBCF05F0080EDBCF06F0D88003AED8904E
:102CC00015E306500A0A12E104C0E9FF05C0EAFF55
:102CD0002D0EEF6E044A052A031E021E011E006C13
:102CE00005E1012A03E1022AD8B4032A0650E56E61
:102CF0000550E56E0450E56E0350E56E0250E56E3A
:102D00000150E56E0050E56E39EC11F0070EE1263A
:102D1000E4CF06F0E4CF05F0E4CF04F0E4CF03F015
:102D2000E4CF02F0E4CF01F0E4CF00F0E4CFD9FF2C
:102D3000120000C0E5FF01C0E5FF02C0E5FF03C0CF
:102D4000E5FF04C0E5FF100E0201195D03E219C2A0
:102D500000F002D0100E006EFC0E04010415046F8A
:102D600000500401056F800E066F050E076F0050BE
:102D70000201195F800E02010E6F050E0F6F00C079
:102D800016F216C200F002011607005024E00EC22F
:102D900000F00FC201F0FDC002F0FEC003F0FFC062
:102DA00004F002C0F6FF03C0F7FF04C0F8FF0900FB
:102DB000F5CF02F00001FD2B03E3FE3F01D0FF2B16
:102DC00000C0E9FF01C0EAFF02C0EFFF02010E3FB1
:102DD00001D00F2BD6D7E4CF04F0E4CF03F0E4CF3B
:102DE00002F0E4CF01F0E4CF00F0120000C0E5FFF4
:102DF00001C0E5FF02C0E5FF03C0E5FF04C0E5FF39
:102E00001F0E0501401542C501F0020A01E03DD048
:102E10000F0E05014415006E800E4415026E015020
:102E200034E1005032E0010E0201186F000E016E15
:102E3000040E036E0050080DF450046EF3CF00F042
:102E40000050012402010E6F045003200F6F025046
:102E500004E0040E0E2701E30F2B05014151030A84
:102E600003E1840E006E07D00250010A02E1006AFD
:102E700002D0880E006E0EC201F00FC202F001C037
:102E8000E9FF02C0EAFF00C0EFFFE4CF04F0E4CFA7
:102E900003F0E4CF02F0E4CF01F0E4CF00F0120041
:102EA00000C0E5FF01C0E5FF0201236B0201246BB6
:102EB00002012E6B0201256B0201266B0201276BBA
:102EC0000201286B0201296B080EB86EE56A2F0E0D
:102ED000E56E3E0EE8EC18F0E652E652020136834B
:102EE000CA6ACA82CA80CB68CA84AB988B909D9A02
:102EF00002012A6BC00E02012A25006E016A000E33
:102F0000012200C0E9FF01C0EAFFEF6AD00E2A25C6
:102F1000006E016A000E012200C0E9FF01C0EAFF55
:102F2000EF6A2A2B100E2A5DE5E3040E02012B6FD7
:102F3000010E02012C6F020E02012D6F9D929F82E5
:102F40009F889F8AF28EE4CF01F0E4CF00F0120058
:102F500011EEFFF021EEFFF0F86AA68EA69CE9685C
:102F60000E0EEA6E0068ED6A0050FDE1C40EF66ECA
:102F7000380EF76E000EF86E0900F5CF05F0090067
:102F8000F5CF06F034D00900F5CF00F00900F5CFF9
:102F900001F00900F5CF02F009000900F5CFE9FFC3
:102FA0000900F5CFEAFF090009000900F5CF03F099
:102FB0000900F5CF04F009000900F6CF07F0F7CFBC
:102FC00008F0F8CF09F000C0F6FF01C0F7FF02C01B
:102FD000F8FF03D00900F5CFEEFF0306FBE204067D
:102FE000F9E207C0F6FF08C0F7FF09C0F8FF0506C1
:102FF000CAE20606C8E29FEC18F0FFD712010002F1
:103000000200001008040A000001010000010A0685
:103010000002020000100100000000010100010098
:1030200009024300020100C032090400000102024B
:1030300001000524001001052401010104240202FD
:1030400005240600010705810308000A09040100A0
:10305000020A000002070502024000000705820282
:1030600040000000040309040E03540065007300CF
:103070007400690021002003550053004200200025
:10308000470065006E006500720069006300200063
:10309000430044004300802500000000080000C0F9
:1030A000E5FF006A6FBE002A0050010A09E0020134
:1030B0001A5106E0006A6DB2002A0050010A01E1CF
:1030C0003BD068A01CD069A01AD06A6A686A9F0EBB
:1030D0006B6E2B0E696E6E6A160E706E006A68B6A5
:1030E000002A0050010A02E16896F8D76D98E0ECDA
:1030F0001BF00201156B030E02011A6F689068AC99
:1031000002D069BC689C68AA0CD069AA0AD0006A7F
:1031100070B0002A0050010A03E1E0EC1BF070904F
:10312000689A68A202D069B2689268A605D069A6BA
:1031300003D0F3EC0EF06896E4CF00F0120034EC0C
:103140001CF08B908B920201036B046B2F0E056FAA
:1031500037EC1BF08B80D08EA29AF28CF28E02019B
:103160001A51050A02E08B82FAD750EC17F00201DF
:10317000235121E1B0EC1BF0006E00501CE050EC3C
:103180001AF0006E0A0A04E1010E0201236F13D047
:103190003F0E0201245DEEE224C201F0242B026AFC
:1031A000C00E0126060E022201C0E9FF02C0EAFF9E
:1031B00000C0EFFFDFD7006A68BC002A0050010A98
:1031C00003E175EC1AF0689C5DEC10F0D0D71200AA
:1031D000D9CFE5FFE1CFD9FF00C0E5FF01C0E5FF92
:1031E00002C0E5FF006E020EDBCF01F0030EDBCF65
:1031F00002F0AC6AAB6A00B0AC8800A202D0AC8C22
:10320000AB8C00A401D0AC8E00A602D0AB8801D05C
:10321000AB8A00A803D0AC84B88601D0B8969E983B
:1032200000AC02D09D8A01D09D9A9E9A00AE02D039
:103230009D8801D09D980250B06E0150AF6E948C65
:10324000948EAC8AAB8EE4CF02F0E4CF01F0E4CFF1
:1032500000F0E4CFD9FF1200D9CFE5FFE1CFD9FFCD
:1032600000C0E5FF01C0E5FF02C0E5FF020ED92462
:10327000006E000EDA20016E800E026E030E002634
:10328000000E012202220250E56E0150E56E005050
:10329000E56E040EDBCFE5FF030EDBCFE5FF020E8C
:1032A000DBCFE5FF02010551E56E0451E56E0351E8
:1032B000E56EB1EC04F0006EF3CF01F0090EE126EB
:1032C00001C0F3FF0050E4CF02F0E4CF01F0E4CFFF
:1032D00000F0E4CFD9FF1200D9CFE5FFE1CFD9FF4D
:1032E00000C0E5FF01C0E5FF02C0E5FF020EDBCF35
:1032F00000F0030EDBCF01F0026A01500201115D04
:1033000002E10050105D07E300500201105F015020
:10331000115B022AF2D702C000F002011C5102E147
:10332000025005E00050E56EA0EC19F0E652E4CF43
:1033300002F0E4CF01F0E4CF00F0E4CFD9FF1200B7
:10334000D9CFE5FFE1CFD9FF00C0E5FF01C0E5FF20
:1033500003C0E5FF020EDBCF00F00A0E005C03E2C3
:10336000300E016E0CD002011B5103E0410E036EC2
:1033700002D0610E036EF60E032603C001F000506A
:1033800001260150E56ED2EC19F0E652010E020161
:103390001C6FE4CF03F0E4CF01F0E4CF00F0E4CF02
:1033A000D9FF1200D9CFE5FFE1CFD9FF00C0E5FF7B
:1033B00001C0E5FF02C0E5FF03C0E5FF020EDBCF61
:1033C00000F000C201F001C202F002C203F000C02E
:1033D000E5FF01C0E9FF02C0F3FF03503FEC1CF022
:1033E0000201002B03E3013F01D0022BE4CF03F0E5
:1033F000E4CF02F0E4CF01F0E4CF00F0E4CFD9FF56
:103400001200D8CFE5FFE0CFE5FFE56EF3CFE5FF93
:10341000F4CFE5FFE9CFE5FFEACFE5FFFACFE5FF1F
:10342000FBCFE5FFA1AA03D04FEC18F0A19AE4CF9F
:10343000FBFFE4CFFAFFE4CFEAFFE4CFE9FFE4CFFC
:10344000F4FFE4CFF3FFE450E4CFE0FFE4CFD8FF94
:10345000100000C0E5FF01C0E5FF02C0E5FF006EFF
:1034600077EC1BF0016E0150FBE1F9C001F00001A7
:10347000F92B026A200E0126040E022201C0E9FF88
:1034800002C0EAFF00C0EFFF400EF95DD8B05BEC70
:103490001CF0E4CF02F0E4CF01F0E4CF00F0120022
:1034A00000C0E5FF01C0E5FFB0EC1BF0006E00506E
:1034B000FBE0FAC000F00001FA2B016A000E0026C2
:1034C000050E012200C0E9FF01C0EAFFEFCF00F0C6
:1034D000040111510001FA5DD8B0EFEC1BF000506F
:1034E000E4CF01F0E4CF00F0120000C0E5FF22C2FB
:1034F00000F00201222B0050C80A13E10201226BE6
:10350000006A8BB2002A0050D880E866D890006A22
:1035100000360050010BE844F46E8B50FD0BF410A4
:103520008B6E0201352B355102E1FF0E3569E4CF78
:1035300000F01200E8AE0AD0F3CFEAFFEE50EECF73
:10354000F3FFEECFF4FFEECFE9FF1200E8BC7EEF11
:103550001CF0E9CFF6FFF3CFF7FFF86E0900F55046
:103560000900F5CFF3FF0900F5CFF4FF0900F5CF0F
:10357000E9FF1200F3CFE5FFF4CFE5FFE9CFE5FF68
:10358000EACFE5FFFACFE5FFFBCFE5FF88EC0DF0D2
:10359000E4CFFBFFE4CFFAFFE4CFEAFFE4CFE9FF9B
:1035A000E4CFF4FFE4CFF3FF1100E8AE08D0F3CF8F
:1035B000EAFFEE50EECFF3FFEECFF4FF1200E8BCCF
:1035C00078EF1CF0E9CFF6FFF3CFF7FFF86E0900B4
:1035D000F5500900F5CFF3FF0900F5CFF4FF120015
:1035E000F2CFEAFFF29EA69EA69CA684E9CFA9FF91
:1035F000E4CFA8FF53EC1CF0F4CFA8FF53EC1CF071
:10360000F6CFA8FF53EC1CF0A694EABEF28E12008F
:10361000F2CFF6FFF29EA69EA69CE9CFA9FFA68058
:10362000A850A92AA680A8CFF3FFA92AA680A8CFD0
:10363000F4FFA92AA680A8CFEAFFF6BEF28E1200F8
:10364000D9CFE5FFE1CFD9FF00C0E5FF020EDBCF08
:1036500000F0610E005C05E37B0E005C02E2010EEF
:1036600001D0E86AE4CF00F0E4CFD9FF1200140ED5
:103670006F6E02011A6B0201156B6DB606D06D6A92
:10368000696A6D86010E02011A6F686A696A69804B
:10369000020E02011A6FA08A1200E8AE06D0F3CF24
:1036A000EAFFEE50EECFF3FF1200E8BC76EF1CF01D
:1036B000E9CFF6FFF3CFF7FFF86E0900F5500900E8
:1036C000F5CFF3FF120000C0E5FF006E00500CE0E4
:1036D00000500401156F040114AD03D0880E146F5F
:1036E00003D0C80E0401146FE4CF00F0120000C034
:1036F000E5FF800E04011415D880E866D890006AB2
:1037000000360050D880E866D890006A0036005035
:10371000E4CF00F01200F2CFF6FFF29EA69EA69C28
:10372000E9CFA9FFA680A850A92AA680A8CFF3FFB9
:10373000A92AA680A8CFF4FFF6BEF28E1200E8AE4A
:1037400004D0F3CFEAFFEE501200E8BC7AEF1CF091
:10375000E9CFF6FFF3CFF7FFF86E0900F55012003E
:10376000040110AF02D0E86A0AD00401115100012F
:10377000FA5D04E3EFEC1BF0E86A01D0010E1200E1
:10378000F2CFF6FFF29EA69EA69CE9CFA9FFA680E7
:10379000A850A92AA680A8CFF3FFF6BEF28E120089
:1037A000F2CFEAFFF29EA69EA69CA684E9CFA9FFCF
:1037B000E4CFA8FF53EC1CF0A694EABEF28E1200F0
:1037C0000201176B100E0401016F400E026F050E0F
:1037D000036F880E0401006F046B6D9812000001E6
:1037E000FA6B400E0401116F040110AD03D0880E76
:1037F000106F03D0C80E0401106F1200E8AE09D09C
:10380000F3CFEAFFE4CFEEFFF4CFEEFFF6CFEEFF0B
:103810001200E8BC7CEF1CF01200D9CFE5FFE1CF2D
:10382000D9FF020EDBCFA9FFA69CA69EA680A850BA
:10383000E4CFD9FF120000C0E5FF006E29EC1AF0BA
:1038400000500A0A02E15BEC1CF0E4CF00F0120029
:10385000F2CFF6FFF29EA69EA69CE9CFA9FFA68016
:10386000A850F6BEF28E12000F0EC112B56A8B6A16
:103870009468FC0E8B169416948494901200E8AE13
:1038800005D0F3CFEAFFE4CFEEFF1200E8BC74EFFF
:103890001CF01200ACA2FED7AE50AB98AB889D8A4C
:1038A0009D988B801200550EA76EAA0EA76EA68259
:1038B000A6B2FED7A94A0001F95163EC1BF0000142
:1038C000F96B12000100E0380000F900000004006C
:1038D0000000ACA2FED7AD6E1200E8CF7FFF120051
:1038E00000000000C96E1200D0EF1BF0C0EF1BF00B
:1038F0008BEF1BF028EF1CF0F0EF1AF008EF1BF035
:020000040030CA
:0E000000200E2000FF8180FFFFFFFFFFFFFFAB
:00000001FF
